S01D000062696E2F6F70656E626C745F73746D3332663330332E7372656397
S3150800000000300020590200089F020008A1020008DB
S31508000010A3020008A5020008A702000800000000C5
S31508000020000000000000000000000000A90200080F
S31508000030AB02000800000000AD020008AF0200088D
S31508000040B1020008B3020008B5020008B7020008AA
S31508000050B9020008BB020008BD020008BF0200087A
S31508000060C1020008C3020008C5020008C70200084A
S31508000070C9020008CB020008CD020008CF0200081A
S31508000080D1020008D3020008D5020008D7020008EA
S31508000090D9020008DB020008DD020008DF020008BA
S315080000A0E1020008E3020008E5020008E70200088A
S315080000B0E9020008EB02000800000000ED02000853
S315080000C0EF0200080000000000000000F10200082E
S315080000D000000000F3020008F5020008F702000815
S315080000E0F9020008FB0200080000000000000000FA
S315080000F000000000000000000000000000000000F2
S3150800010000000000000000000000000000000000E1
S315080001100000000000000000FD020008FF020008C1
S3150800012000000000000000000000000000000000C1
S3150800013000000000000000000000000000000000B1
S315080001400103000803030008000000000000000087
S315080001500000000000000000000000000000000091
S315080001600000000000000000000000000000000081
S315080001700000000000000000000000000000000071
S31508000180000000000503000810B5054C237833B9B4
S31508000190044B13B10448AFF300800123237010BD4C
S315080001A09C00002000000000C01A0008084B10B58B
S315080001B01BB108490848AFF300800848036803B92B
S315080001C010BD074B002BFBD0BDE81040184700BFF9
S315080001D000000000A0000020C01A00089C000020B3
S315080001E000000000154B002B08BF134B9D46A3F5D6
S315080001F0803A00218B460F461348144A121A01F01A
S315080002000BFC0F4B002B00D098470E4B002B00D051
S3150800021098470020002104000D000D48002802D050
S315080002200C48AFF3008001F0D1FB2000290000F054
S31508000230FBF801F0B7FB00BF000008000030002003
S3150800024000000000000000009C000020A805002017
S3150800025000000000000000000649074A074B9A42C2
S31508000260BEBF51F8040B42F8040BF8E70448804770
S3150800027004480047CC1A0008000000209C00002013
S315080002803D050008E50100081F49204A002301E052
S3150800029041F8043B9142FBD300F0C6F8FEE7FEE7BF
S315080002A0FEE7FEE7FEE7FEE7FEE7FEE7FEE7FEE718
S315080002B0FEE7FEE7FEE7FEE7FEE7FEE7FEE7FEE708
S315080002C0FEE7FEE7FEE7FEE7FEE7FEE7FEE7FEE7F8
S315080002D0FEE7FEE7FEE7FEE7FEE7FEE7FEE7FEE7E8
S315080002E0FEE7FEE7FEE7FEE7FEE7FEE7FEE7FEE7D8
S315080002F0FEE7FEE7FEE7FEE7FEE7FEE7FEE7FEE7C8
S31508000300FEE7FEE7FEE700009C000020A8050020A7
S315080003102DE9F04182B001214FF4802000F07AFCEB
S315080003204FF00808CDF8008001248DF80440002518
S315080003308DF8065003268DF805608DF80750394F5D
S315080003406946384600F04CFA4146384600F09AFAB3
S3150800035021464FF4003000F05DFC8DF804508DF80E
S3150800036007404FF40073009369464FF0904000F041
S3150800037037FA21464FF4003000F05AFC21464FF474
S31508000380003000F047FC072202214FF0904000F0B1
S315080003907BFA07220F214FF0904000F075FA8DF88E
S315080003A006508DF8074002278DF804700423009341
S315080003B08DF8056069464FF0904000F011FA8DF807
S315080003C004704FF40043009369464FF0904000F0E4
S315080003D007FA21464FF4003000F01CFC09220B21D5
S315080003E04FF0904000F050FA09220C214FF090404F
S315080003F000F04AFA4FF4C05300938DF804708DF854
S3150800040005608DF806508DF8074069464FF0904014
S3150800041000F0E6F921464FF0007000F009FC02B042
S31508000420BDE8F0810004004808B5FFF771FF00F049
S315080004303DFC00F049FCFCE708B500F045F84FF430
S3150800044000714FF0904000F013FA034600B1012303
S31508000450184608BD08B5642000F006F808BD00BFB8
S3150800046008B500F007F808BD014B1880704700BFB3
S31508000470BC00002008B501F03BFA0F4B1B689842F8
S3150800048018D30E4B1B783BB901220C4B1A70082166
S315080004900B4800F0F5F906E00022084B1A7008210F
S315080004A0074800F0EFF901F023FA064B1B881844B9
S315080004B0014B186008BD00BFB8000020BE00002030
S315080004C000040048BC00002008B50821014800F0D7
S315080004D0D9F908BD000400481222164B1A60A3F584
S315080004E080535A685A605A685A605A6842F4806259
S315080004F05A605A6822F47C125A605A6842F46012AA
S315080005005A601A6842F080721A600B4B1B6813F027
S31508000510007FFAD0084B5A6822F003025A605A68DC
S3150800052042F002025A60044B5B6803F00C03082B86
S31508000530F9D17047002002400010024010B5174C50
S31508000540D4F8883043F47003C4F88830144B1A681A
S3150800055042F001021A605968124A0A405A601A683B
S3150800056022F0847222F480321A601A6822F48022F9
S315080005701A605A6822F4FE025A60DA6A22F00F02FA
S31508000580DA62196B084A0A401A6300229A60FFF772
S31508000590A3FF4FF00063A36010BD00BF00ED00E0AD
S315080005A0001002400CC07FF8CCFC00FFFEE700BF3D
S315080005B0054B1B6913F0800F05D0034B034A5A609D
S315080005C002F188325A6070470020024023016745CD
S315080005D0024A136943F08003136170470020024002
S315080005E0014BD860704700BF002002400B4BDB6808
S315080005F013F0010F0BD1094BDB6813F0100F08D16C
S31508000600064BDB6813F0040F05D003207047012062
S315080006107047022070470420704700BF0020024040
S3150800062010B50446FFF7E2FF02E0FFF7DFFF013CE3
S31508000630012801D1002CF8D104B9052010BD00BF4E
S3150800064038B505464FF43020FFF7EAFF042811D1E4
S31508000650094C236943F0020323616561236943F06A
S31508000660400323614FF43020FFF7DAFF236923F0B4
S315080006700203236138BD00BF0020024030B583B0B5
S3150800068005460C46002301934FF43020FFF7C8FFB8
S31508000690042820D1114A136943F001031361A3B258
S315080006A02B804FF43020FFF7BBFF04280ED102350C
S315080006B00195019B240C1C804FF43020FFF7B0FFF6
S315080006C0064A136923F00103136104E0034A136918
S315080006D023F00103136103B030BD00BF00200240C0
S315080006E030B599B004460D46036823F0010303604C
S315080006F0436823F440528B6813434360036823F42A
S31508000700B05222F00C024968EB6819432B690B4377
S3150800071013430360836823F440726B691343836051
S3150800072001A800F0C9F81C4B9C4201D10F9A0FE0B2
S315080007301A4B9C4201D1109A0AE0194B9C4201D1EE
S31508000740119A05E0174B9C4201D1129A00E0139AC0
S31508000750236813F4004F06D052002968B2FBF1F360
S3150800076001FB132204E02968B2FBF1F301FB132213
S315080007702968B2EB510F00D30133226812F4004FF7
S3150800078006D0C3F3420223F00F031B041B0C1343CA
S315080007909BB2A38119B030BD003801400044004027
S315080007A000480040004C004021B1036843F00103B3
S315080007B003607047036823F001030360704700BFB6
S315080007C0C1F3080101857047808CC0F308007047A3
S315080007D0C3690B4201D0012070470020704700BF53
S315080007E070B400233FE001229A400C68A24339D135
S315080007F00A79013AD2B2012A1CD885685A0003241C
S31508000800944025EA0404846085684C7904FA02F267
S315080008102A4382608488A5B29AB20124944025EAC4
S31508000820040484808588ADB28C7904FA02F292B207
S315080008302A43828004685A00032505FA02F624EA48
S315080008400604046006680C79944034430460C4685E
S315080008509EB27600B54024EA0505CC7904FA02F280
S315080008602A43C26001330F2BBDD970BC704700BF45
S31508000870038A194201D0012070470020704700BF43
S31508000880816170470185704730B401F007039B000A
S315080008909A40C908083150F821400F2505FA03F394
S315080008A024EA030340F8213050F821301A4340F86F
S315080008B0212030BC704700BFF0B5A04B5B6803F041
S315080008C00C03042B06D0082B08D003BB9C4B0360F3
S315080008D000241FE09A4B036000241BE0974B5C68DA
S315080008E05A68C4F38344A31C12F4803F03D1954C81
S315080008F004FB03F409E0914AD26A02F00F020132BE
S315080009008F4CB4FBF2F404FB03F4046002E08C4B56
S3150800091003600024894D6B68C3F30313DFF828E2EC
S315080009201EF80370FFB2026822FA07F3436069688B
S31508000930C1F302211EF80110C9B223FA01F1816040
S315080009406E68C6F3C2261EF80660F6B2F340C360A8
S31508000950ED6A2D0905F00F0CDFF8F0E13EF81CE012
S315080009601FFA8EFE15F0100F06D0BEF1000F03D049
S31508000970B4FBFEF5056100E00261704DED6A6D0A93
S3150800098005F00F0CDFF8C4E13EF81CE01FFA8EFEF6
S3150800099015F0100F06D0BEF1000F03D0B4FBFEF51C
S315080009A0456100E04261654D2D6B15F0100F02D1CF
S315080009B0634D856100E08261604D2D6B15F0200F57
S315080009C002D15F4DC56100E0C2615C4D2D6B15F02B
S315080009D0400F02D15A4D056200E00262574D2D6B59
S315080009E015F4807F06D0944204D1B74202D165003F
S315080009F0456200E04362514D2D6B15F4805F06D0C9
S31508000A00944204D1B74202D16500856200E0836250
S31508000A104A4D2D6B15F4007F06D0944204D1B74297
S31508000A2002D16500C56200E0C362444D2D6B15F422
S31508000A30806F06D0944204D1B74202D16500C564DE
S31508000A4000E0C3643D4D2D6B15F4006F06D094424B
S31508000A5004D1B74202D16500056500E00365374D4C
S31508000A602D6B15F4005F06D0944204D1B74202D12B
S31508000A706500456500E00365304D2D6B15F4004FA4
S31508000A8006D0944204D1B74202D16400846500E0DE
S31508000A9083652A4B1B6B13F0030F01D1816319E0A1
S31508000AA0264B1B6B03F00303012B01D1826311E074
S31508000AB0224B1B6B03F00303022B03D14FF40043B5
S31508000AC0836307E01D4B1B6B03F00303032B01D164
S31508000AD01B4B8363194B1B6B13F4403F01D1C16356
S31508000AE01CE0164B1B6B03F44033B3F5803F01D172
S31508000AF0C26313E0114B1B6B03F44033B3F5003F9D
S31508000B0003D14FF40043C36308E00C4B1B6B03F49B
S31508000B104033B3F5403F01D1094BC363074B1B6B09
S31508000B2013F4402F01D1016426E0044B1B6B03F438
S31508000B304023B3F5802F0BD102641DE0001002405C
S31508000B4000127A0000093D00200000200000002065
S31508000B502E4B1B6B03F44023B3F5002F03D14FF440
S31508000B600043036408E0294B1B6B03F44023B3F5E9
S31508000B70402F01D1264B0364244B1B6B13F4401FF3
S31508000B8001D141641CE0214B1B6B03F44013B3F500
S31508000B90801F01D1426413E01C4B1B6B03F4401306
S31508000BA0B3F5001F03D14FF40043436408E0174B25
S31508000BB01B6B03F44013B3F5401F01D1144B436478
S31508000BC0124B1B6B13F4400F01D18164F0BD0F4B20
S31508000BD01B6B03F44003B3F5800F01D18264F0BDAB
S31508000BE00A4B1B6B03F44003B3F5000F03D14FF414
S31508000BF000438364F0BD054B1B6B03F44003B3F558
S31508000C00400F01D1024B8364F0BD00BF00100240C3
S31508000C1000127A0021B1054B5A6910435861704792
S31508000C20024A536923EA00005061704700100240E7
S31508000C3021B1054BDA691043D8617047024AD36976
S31508000C4023EA0000D06170470010024008B500F0A2
S31508000C50B5F8FCE708B500F0A9F8012810D0094B4B
S31508000C601B78012B0CD100F043FE074B1B6803F5DC
S31508000C70FA73984204D30022024B1A7000F044FE1D
S31508000C8008BD00BFBF000020C000002008B5012233
S31508000C90044B1A7000F02CFE034B1860FFF7DAFFBE
S31508000CA008BD00BFBF000020C000002008B500F046
S31508000CB027FE00F07FF800F0FBFD00F051FE00F083
S31508000CC00DF8FFF7E3FF08BD08B500F077F800F068
S31508000CD001FE00F013F8FFF7BDFF08BD10B500F0E0
S31508000CE0DBF900F093FA044C0123237000F0C0FBF3
S31508000CF00023237010BD00BF3000002008B50B4844
S31508000D0000F052FB012805D10122094B1A70074849
S31508000D1000F0E0F9054800F0EDFB012805D10022B6
S31508000D20034B1A70014800F0D5F908BDC40000202D
S31508000D3030000020704700BF38B504460D46084B02
S31508000D401B78012B02D1C9B200F0E4FA044B1B78D8
S31508000D501BB9E9B2204600F0A5FB00F0B3F938BD8F
S31508000D6030000020074B1B78022B05D0032B05D03B
S31508000D70012B05D04020704700207047002070479F
S31508000D800820704730000020074B1B78022B05D03F
S31508000D90032B05D0012B05D0402070470020704753
S31508000DA000207047082070473000002008B500F082
S31508000DB081F908BD08B5FFF74DFB08BD08B5FFF773
S31508000DC04FFB08BD10B4002304E010F8011B0B44C8
S31508000DD0DBB221464C1E0029F7D1136001205DF8CD
S31508000DE0044B70470022014B5A70704704010020DB
S31508000DF0034BFE22DA7018710222A3F844207047CA
S31508000E000401002010B5054C00232370FFF7EAFF04
S31508000E10FF23E3700123A4F8443010BD0401002029
S31508000E20064BFF22DA7000221A71597859719A71A5
S31508000E30DA711A720622A3F84420704704010020CA
S31508000E4008B50020FFF7D4FF08BD00BF084BFF22F6
S31508000E50DA70084A9A6400221A715A719A7107213F
S31508000E60D9711A725A729A720822A3F844207047E6
S31508000E7004010020401A0008044BFF22DA70426879
S31508000E809A640122A3F84420704700BF0401002099
S31508000E9010B5084CFF23E370E21D4168A06CFFF70C
S31508000EA091FF207100236371A3710823A4F84430CD
S31508000EB010BD00BF0401002008B53120FFF798FFD8
S31508000EC008BD00BF38B5084CFF23E370002525711F
S31508000ED06571FFF747FFA071E571257265720723F3
S31508000EE0A4F8443038BD00BF0401002038B5FFF728
S31508000EF079FF0E4C01252570FF23E370102323711B
S31508000F0000236371FFF72EFFA071FFF73DFFE07125
S31508000F10FFF73AFFC0F3072020726572A57208230F
S31508000F20A4F8443000F01CFD38BD00BF04010020C1
S31508000F3038B505464478FFF715FF0138844203DDC6
S31508000F402220FFF755FF38BD084C6A78A16C201D92
S31508000F5000F0F6FCFF23E3706B78A26C1344A364DD
S31508000F606B780133A4F8443038BD00BF0401002073
S31508000F7038B504464578FFF7F5FE0138854203DDA6
S31508000F802220FFF735FF38BD6168084DA9646278ED
S31508000F90281D00F0D5FCFF23EB706378AA6C134478
S31508000FA0AB6463780133A5F8443038BD04010020EA
S31508000FB038B505460D4B9C6CFFF7D4FE6A1C411EDE
S31508000FC0204600F0D1FC18B93120FFF711FF38BDD3
S31508000FD0064CFF23E370FFF7C5FE0138A36C1844DF
S31508000FE0A0640123A4F8443038BD00BF04010020E2
S31508000FF038B504464578FFF7B5FE0238854203DD65
S315080010002220FFF7F5FE38BD0F4BFF22DA700122CA
S31508001010A3F84420617831B900F0B6FC90B93120C4
S31508001020FFF7E6FE38BDA21C074B986C00F09CFC47
S3150800103018B93120FFF7DCFE38BD6378024A916C97
S315080010400B44936438BD00BF0401002008B541680D
S31508001050074B986C00F08CFC18B93120FFF7C8FED6
S3150800106008BD034BFF22DA700122A3F8442008BD0D
S315080010700401002008B500F047FC034BFF22DA7094
S315080010800122A3F8442008BD0401002008B589B24E
S31508001090FFF752FE08BD00BF054B00221A709A647E
S315080010A083F84320A3F844209A705A70704700BF0B
S315080010B004010020024B187800B10120704700BFD8
S315080010C0040100200022024B83F84320704700BF2A
S315080010D00401002008B50378FF2B02D1FFF706FFAD
S315080010E050E0334A1278012A60D1C93B352B46D8DD
S315080010F0DFE803F03345454245453F363C3945452B
S315080011004545454545454545454545454545454581
S315080011104545454545454545454545454545241EB9
S315080011201B2145454527452A2D30FFF701FF29E0B4
S31508001130FFF71EFF26E0FFF79FFE23E0FFF7A8FE56
S3150800114020E0FFF783FE1DE0FFF77AFE1AE0FFF7BF
S3150800115067FE17E0FFF756FE14E0FFF729FF11E0D8
S31508001160FFF746FF0EE0FFF7ADFE0BE0FFF76EFF59
S3150800117008E0FFF77FFF05E0FFF79EFE02E020206C
S31508001180FFF736FE0A4B93F84330012B02D11020A5
S31508001190FFF72EFE064BB3F94410002906DD184664
S315080011A0012380F843300330FFF770FF08BD00BF06
S315080011B004010020F0B5002422E0134D15F814E0D0
S315080011C005EB44056F780EEB070606FB00064FF4A1
S315080011D0FA4595FBF6F506FB05F5B5F5FA4F0DD17B
S315080011E095FBF6F6B6B20E80013EB6B2B6F5806F3E
S315080011F004D282F800E01F700120F0BD0134E4B289
S31508001200112CDAD90020F0BD701A000800B583B099
S3150800121001AB0DF105020DF106014FF4FA70FFF767
S31508001220C9FF012803D0E2213848FFF70FFD384BE4
S3150800123000225A611A6842F400421A6001E0FFF778
S31508001240BDFD334B1B6813F4004FF8D1304B1A68B9
S3150800125022F002021A601A6842F001021A6001E0DE
S31508001260FFF7ACFD2A4B5B6813F0010FF8D09DF829
S3150800127005305A1E9DF80430013B1B0543EA02431C
S31508001280BDF80620013A1343214AD361136823F0B7
S315080012900103136001E0FFF791FD1D4B5B6813F036
S315080012A0010FF8D11A4BD3F8002242F00102C3F815
S315080012B00022D3F81C2222F00102C3F81C22D3F81C
S315080012C00C2242F00102C3F80C220022C3F8402285
S315080012D0C3F84422D3F8042222F00102C3F80422F8
S315080012E0D3F8142222F00102C3F81422D3F81C22E0
S315080012F042F00102C3F81C22D3F8002222F00102B0
S31508001300C3F8002203B05DF804FB00BF481A0008C2
S315080013100064004038B504460D46214B9B6813F01F
S31508001320806F04D140F221111E48FFF78FFC1C4B39
S31508001330D3F8802102F00102C3F88021D3F8802176
S3150800134042F07C4242F40012C3F88021C3F884516B
S31508001350E178A278120442EA0162617842EA01223F
S3150800136021780A43C3F88821E179A279120442EA6E
S315080013700162617942EA012221790A43C3F88C2184
S31508001380D3F8802142F00102C3F8802101E0FFF77B
S3150800139015FD034B9B6813F0806FF8D038BD00BF6E
S315080013A000640040481A00081B4BDB6813F0030F63
S315080013B02FD0194BD3F8B02140F26763B3EB525FD5
S315080013C020D1154BD3F8B8210270D3F8B821120AE8
S315080013D04270D3F8B821120C8270D3F8B821120ED5
S315080013E0C270D3F8BC210271D3F8BC21120A42712B
S315080013F0D3F8BC21120C8271D3F8BC311B0EC37111
S31508001400012000E00020044AD36843F02003D3609B
S3150800141070470020704700BF0064004010B50446BE
S3150800142080210948FFF7D4F958B121460648FFF745
S31508001430C7F980210448FFF7CBF90028F9D0012025
S3150800144010BD002010BD00BF0044004010B5044682
S3150800145020210648FFF7BCF9012805D10348FFF704
S31508001460B3F92070012010BD002010BD00440040D3
S3150800147010B586B04FF4614300930023019302939D
S31508001480039305930C230493054C69462046FFF7FE
S3150800149027F901212046FFF787F906B010BD00BFDE
S315080014A00044004070B506460D46402903D975210B
S315080014B00F48FFF7CBFB2846FFF7B0FF012803D0FC
S315080014C079210B48FFF7C2FB00240CE0FFF776FCF6
S315080014D0305DFFF7A3FF012803D082210448FFF7F8
S315080014E0B5FB0134A4B2ABB29C42EFD370BD00BFCA
S315080014F0941A000838B5224B1C789CB92148FFF786
S31508001500A5FF01283AD11F4B1B78002B31D000F0DC
S31508001510EFF91D4B186000221C4B1A700122184B5C
S315080015201A702BE00546194B1B78013315481844E9
S31508001530FFF78CFF0446012810D1144B1A780132A4
S31508001540D2B21A700F4B1B789A4214D1104928460A
S3150800155000F0F6F900220A4B1A700FE000F0C8F9FD
S31508001560094B1B686433984207D90024044B1C7046
S3150800157004E01C4602E0002400E00024204638BDB2
S315080015809901002058010020500100205401002034
S315080015905901002008B5C1F3080353B903689942F5
S315080015A009D040F8041B4FF4007200F0C9F9012075
S315080015B008BD002008BD012008BD00BF2DE9F04187
S315080015C00746FEF7F5FF3420FFF70AF8FFF70EF88F
S315080015D0012815D100241BE03E68A30006EB03088A
S315080015E03B445D68FFF7EAFB29464046FFF746F8A5
S315080015F004280AD156F824309D4208D1013400E067
S3150800160000247F2CE8D9012402E0002400E000240D
S31508001610FEF7DEFF2046BDE8F08100BF38B50D466F
S315080016200B4B984207D004460A4B994205D0FFF760
S31508001630C5FF18B908E0084C00E0054C29462046C5
S31508001640FFF7A8FF10B938BD002038BD204638BDC1
S315080016509C01002000200008A00300202DE9F0418D
S3150800166006460C4617461D4621F4FF7828F0010861
S315080016700368B3F1FF3F04D14146FFF78BFF0346EA
S3150800168030B33368984505D041463046FFF7C6FF64
S315080016900646D0B13368E41A34440434FFF78EFBA7
S315080016A0331DE31AB3F5007F07D308F500713046FA
S315080016B0FFF7B4FF064650B1041D17F8013B04F8BE
S315080016C0013B013DEAD1012302E0002300E00023AB
S315080016D01846BDE8F08100BF4FF0FF33024A136099
S315080016E0024A1360704700BFA00300209C01002037
S315080016F00E4B984216D910B54318013B0C4CA34221
S3150800170012D80B46014620F4FF7020F00100094C60
S31508001710A04203D10848FFF7A1FF10BD0748FFF70D
S315080017209DFF10BD00207047002010BDFF1F000858
S31508001730FFFF0008002000089C010020A0030020ED
S3150800174070B520F4FF6525F007051A4B9D422DD983
S315080017504318013B184A93422AD8401B0144C1F357
S31508001760CF26C1F30A0109B10136B6B2FEF720FF4A
S315080017703420FEF735FFFEF739FF01280CD1002487
S3150800178010E0FFF71BFB05EBC420FEF759FF042802
S3150800179007D10134A4B200E00024A642F1D80124FE
S315080017A000E00024FEF714FF204670BD002070BD3F
S315080017B0002070BDFF1F0008FFFF0008114B1B68C3
S315080017C0B3F1FF3F18D000B583B00E4B59689A683D
S315080017D01144DA6811441A6911445A6911449A691C
S315080017E01144DA698B185B4202AA42F8043D0421C7
S315080017F00548FFF77DFF01E00120704703B05DF85B
S3150800180004FB00BF9C010020882100080D4B1A68C4
S3150800181004331B6813440C4A126813440B4A1268B3
S3150800182013440B4A11680B44043212681A44094BD4
S315080018301B681344084A1268D34201D10120704735
S315080018400020704700200008082000080C20000827
S3150800185010200008182000088821000808B50D4B3C
S315080018601B68B3F1FF3F04D00A48FFF7A7FE0346FB
S3150800187068B1094B1B68B3F1FF3F05D00648FFF76F
S315080018809DFE034610B902E0012300E00123184635
S3150800189008BD00BF9C010020A00300200048704737
S315080018A0002000080022014B1A60704710E000E093
S315080018B008B5FFF7F7FF054B4FF6FF125A600022EF
S315080018C09A6005211960024B1A6008BD10E000E015
S315080018D0A4050020044B1B6813F4803F03D0034A79
S315080018E0136801331360704710E000E0A405002078
S315080018F008B5FFF7EFFF014B186808BDA4050020DF
S3150800190008B500F04BF808BD10B500F035F8A0B1E1
S31508001910FEF792FD88B1FFF70DFAFFF7C3FF00F057
S315080019202FF820F0604020F07F00044B186000F08C
S3150800193027F8446800F034F8A04710BD08ED00E029
S3150800194070B508E0461C4D1C0B780370FFF736FA95
S31508001950224630462946531E9CB2002AF2D170BD53
S3150800196008B5FFF7B9FE08BD08B5FFF7C1FE08BD03
S3150800197008B5FFF7E5FE08BD08B5FFF747FF08BD40
S3150800198008B5FFF78BFF08BD08B5FFF717FF034635
S3150800199010B1FFF763FF0346184608BD72B67047D5
S315080019A062B6704708B5074B044613B10021AFF37A
S315080019B00080054B1868836A03B198472046FEF7EE
S315080019C0F5FD00BF00000000BC1A000870B50E4BFC
S315080019D00E4CE41AA41000251E46A54204D056F85B
S315080019E0253098470135F8E700F01EF8084C094BF2
S315080019F0E41AA41000251E46A54204D056F8253040
S31508001A0098470135F8E770BD94000020940000203F
S31508001A10980000209400002002440346934202D016
S31508001A2003F8011BFAE77047F8B500BFF8BC08BC15
S31508001A309E467047F8B500BFF8BC08BC9E4670477E
S31508001A404F70656E424C54002E2E2F2E2E2F2E2EA2
S31508001A502F536F757263652F41524D434D345F5353
S31508001A60544D333246332F63616E2E6300000000F7
S31508001A7005020602060307030803090309040A0404
S31508001A800B040C040C050D050E050F050F061006B4
S31508001A90100710082E2E2F2E2E2F2E2E2F536F7531
S31508001AA07263652F41524D434D345F53544D333263
S31508001AB046332F756172742E6300000034000020CF
S30908001AC00000000014
S30D08001AC420E7FF7F0100000086
S31508001ACC010002000400060008000A000C001000C1
S31508001ADC200040008000000100000000000000000B
S31508001AEC00000000010203040102030406070809AA
S31508001AFC04000000000000000000000000000000C8
S31508001B0C00000000000000000000000000000000BB
S31508001B1C00000000000000000000000000000000AB
S31508001B2C000000000000000000000000000000009B
S31508001B3C000000000000000000000000000000008B
S31508001B4C000000000000000000000000000000007B
S31108001B5C00000000AD0100088901000827
S70508000000F2
